:100245001110C0F3A4A1938988E380818298CCB072
:030255008C8E008C
:0E0003008B388A39893A8F3E8E3D8D3C8C3B7E
:1000110090000C120682AB3EAA3DA93CA83B1203FC
:10002100518F468E458D448C43AB38E53A2404F913
:10003100E43539FAC003C002C001120662AB3EAA20
:100041003DA93CA83B120260D001D002D0031206A8
:10005100B2AB38AA39A93A9000041206829000087E
:100061001206CC1203518F4E8E4D8D4C8C4BAB38FA
:10007100AA39A93A120662AB42AA41A940A83F1285
:10008100025CAB38AA39A93A9000101206CC1203CF
:10009100518F4A8E498D488C47AF42AE41AD40AC3D
:1000A1003FAB38AA39A93A1206B2AF4AAE49AD48B8
:1000B100AC47AB46AA45A944A843120260AB4EAA7D
:0800C1004DA94CA84B1202608E
:0100C9002214
:1000CA001206FC000000009000041207160000004F
:1000DA000090000812071638D1B71790000C1207C3
:1000EA001642CC00009000101207160000000022F1
:1000FA00750B00750A00750900750800750F007503
:09010A000E00750D00750C0022B9
:100113007B007A0079207841AF0FAE0EAD0DAC0CA9
:1001230012045AA804A905AA06AB07AF0BAE0AAD81
:1001330009AC0812025C8F3B8E3A8D398C38AB0FB9
:10014300AA0EA90DA80CC000C001C002C0037FCD38
:100153007ECC7DCC7C3DAB3BAA3AA939A8381203AF
:1001630051D003D002D001D0001202608F0F8E0E47
:100173008D0D8C0C7F007E007D007C00AB0FAA0EE2
:10018300A90DA80C1204F3500A7F007E007D007CA9
:10019300008008AF0FAE0EAD0DAC0C8F0F8E0E8D21
:0301A3000D8C0CB4
:0101A6002236
:1001A7007B007A0079241200CA1200FA7F007E00D1
:1001B7007D827C42AB0FAA0EA90DA80C12025C85AA
:1001C7000F42850E41850D40850C3F7B007A0079F3
:1001D7002412000312059E8F21E521C394005005C8
:1001E700E4F521800AE521D394644003752164ACCA
:1001F70021E412056A7BEC7A517938783E12035173
:100207008F0B8E0A8D098C08AF0FAE0EAD0DAC0C9F
:1002170012059E8E228F237C007D0A12061E741003
:100227002FF8E6F580AE22AF237C007D0A12061E6A
:0D02370074102DF8E6F5A01201130201B3BA
:010244002297
:1002590002060AE86480F8E933E83360110460F0C3
:10026900ED33EC337009E8FCE9FDEAFEEBFF22040B
:1002790060DED3EB9FEA9EE99DE8C2E78CF0C2F706
:1002890095F0400CE8CCF8E9CDF9EACEFAEBCFFBD2
:100299001205D585D0F05804700320D5B3E8047051
:1002A900075002B2D502061492D5EC0460F7E4CCEB
:1002B900C0E0C398F8603B94186008400DD0E0FB9B
:1002C9000205ECE4FBFAC9FC8028E830E406E4C93D
:1002D900FBE4CAFCE830E305E4C9CACBFCE85407EF
:1002E9006010F8C3E913F9EA13FAEB13FBEC13FCFA
:1002F900D8F130F52FC3E49CFCEF9BFFEE9AFEED9D
:1003090099FDD0E0FBEF4E4D4C701222DB03020643
:1003190011EC2CFCEF33FFEE33FEED33FDED30E74E
:10032900EB0205ECEF2BFFEE3AFEED39FDD0E0FBD9
:1003390050130BBB0003020614ED13FDEE13FEEF81
:0803490013FFEC13FC0205ECAC
:10035100EC4D6011E8497017ED33EC3304600DE4A6
:10036100FCFFFEFD22E933E8330470F802060A12AD
:1003710005D558046009E4CC2481500628500902AF
:100381000614284003020611C0E0EB4A7044B9800C
:1003910006D0E0FB020600EF4E701CBD8008EBFFAB
:1003A100EAFEE9FD80EBE98DF0A4FEE5F002043AF6
:1003B100E9CDF9EAFEEBFFEF89F0A4FCE5F0CE8987
:1003C100F0A42EFFE435F0CD89F0A42DFEE435F044
:1003D1008067EF4E7005BD80D780C3EF8BF0A4AC72
:1003E100F0EE8BF0A42CFCE435F0F8EF8AF0A42CAD
:1003F100E5F038FCE433CB8DF0A42CFCE5F03BF8C0
:10040100EE8AF0A42CFCE5F038F8E433CF89F0A4AF
:100411002CFCE5F038CF3400CE89F0A42FFFE5F0B5
:100421003EFEE433C98DF0A42EFEE5F039CD8AF00D
:10043100A42FFFE5F03EFEE43DFD33D0E0FB500785
:100441000BBB000F020614EC2CFCEF33FFEE33FE66
:06045100ED33FD0205EC95
:10045700020614EC5D046005E85904700302060AFD
:100467001205D5580460F6EC4860F2EC7004FDFE06
:10047700FF22C82481C85007C39850060206119866
:1004870050CEF582E9294B4A7005AB82020600750A
:10049700F0007C1A7880C3EF9BEE9AED99400DC36C
:1004A700EF9BFFEE9AFEED99FDE842F0DC23ACF0FE
:1004B700D0E0FFD0E0FED0E0FDAB8220E7101BEBE1
:1004C70060BAEC2CFCEF33FFEE33FEED33FD020593
:1004D700ECE803F830E705C0F075F000EF2FFFEE0A
:0C04E70033FEED33FD40B830E7C280AAC0
:1004F30074F8CC6480CCC86480C8F582046043C3BC
:10050300EB9FF5F0EA9E42F0E99D42F0E89C45F04E
:1005130060305018E5825FFFE582F42B5582FB5073
:10052300210ABA001D09B90019088016E5825BFB90
:10053300E582F42F5582FF50090EBE00050DBD0064
:10054300010CC3EB9FF5F0EA9E42F0E99D42F0E80F
:0D0553009C45F06007CC4820E701B3EC2286
:1005600075F020800E75F010800575F0087D007E16
:10057000007F003392D530D503120654EC3340107F
:10058000EF33FFEE33FEED33FDEC33FCD5F0ED221F
:0E059000E5F0247EA2D513CC92E7CDCEFF225B
:10059E00EDD2E7CD33EC3392D524814006E4FFFE55
:1005AE00FDFC22FCE4CFCECDCC24E0501174FF80B4
:1005BE00EDC3CC13CCCD13CDCE13CECF13CF047051
:0705CE00F030D5DE020654F7
:1005D500E9D2E7C933E833F892D5EDD2E7CD33EC6C
:0705E50033FC5002B2D522E5
:1005EC00EC30E7100FBF000C0EBE00080DBD000470
:1005FC000BEB6014A2D5EB13FCED92E7FD2274FF1C
:10060C00FCFDFEFF22E480F8A2D574FF13FC7D8074
:02061C0080F06C
:0300000002088073
:0C088000787FE4F6D8FD75814E0208C7B1
:10061E00C2D5EC30E709B2D5E4C39DFDE49CFCEEF7
:10062E0030E715B2D5E4C39FFFE49EFE12073AC32E
:10063E00E49DFDE49CFC800312073A30D507C3E429
:06064E009FFFE49EFE2266
:0E065400C3E49FFFE49EFEE49DFDE49CFC22B7
:10066200BB010789828A8302079B5005E9F80207CA
:100672008FBBFE05E9F80207A789828A830207B3C6
:10068200BB010DE58229F582E5833AF58302079BDA
:100692005007E92582F802078FBBFE07E92582F899
:1006A2000207A7E58229F582E5833AF5830207B3BB
:1006B200BB010789828A830208055005E9F802070F
:0A06C200F9BBFE05E9F80208112259
:1006CC00BB010DE58229F582E5833AF5830207D05B
:1006DC005007E92582F80207C3BBFE07E92582F81B
:1006EC000207DCE58229F582E5833AF5830207E906
:1006FC00BB010789828A830208365005E9F8020893
:0A070C001DBBFE05E9F80208672294
:10071600BB010DE58229F582E5833AF583020836A9
:100726005007E92582F802081DBBFE07E92582F875
:04073600020867222C
:10088C000201A7E493A3F8E493A34003F68001F2DA
:10089C0008DFF48029E493A3F85407240CC8C3336D
:1008AC00C4540F4420C8834004F456800146F6DF3C
:1008BC00E4800B0102040810204080900245E47E85
:1008CC00019360BCA3FF543F30E509541FFEE49331
:1008DC00A360010ECF54C025E060A840B8E493A3F8
:1008EC00FAE493A3F8E493A3C8C582C8CAC583CA23
:1008FC00F0A3C8C582C8CAC583CADFE9DEE780BEDB
:0102580000A5
:10073A00BC000BBE0029EF8DF084FFADF022E4CCA3
:10074A00F875F008EF2FFFEE33FEEC33FCEE9DEC6C
:10075A00984005FCEE9DFE0FD5F0E9E4CEFD22EDB2
:10076A00F8F5F0EE8420D21CFEADF075F008EF2FFC
:10077A00FFED33FD4007985006D5F0F222C398FDED
:05078A000FD5F0EA228A
:0C078F00E6FC08E6FD08E6FE08E6FF2296
:0C079B00E0FCA3E0FDA3E0FEA3E0FF22D1
:0C07A700E2FC08E2FD08E2FE08E2FF228E
:1007B300E493FCA3E493FDA3E493FEA3E493FF2259
:0D07C300E6FB08E6F908E6FA08E6CBF822A6
:0C07D000E0F8A3E0F9A3E0FAA3E0FB22AC
:0D07DC00E2FB08E2F908E2FA08E2CBF8229D
:1007E900E493F8A3E493F9A3E493FAA3E493FB2233
:0C07F900ECF608EDF608EEF608EFF6222C
:0C080500ECF0A3EDF0A3EEF0A3EFF02266
:0C081100ECF208EDF208EEF208EFF22223
:10081D00D083D082E493F608740193F608740293A2
:09082D00F608740393F6740473D9
:10083600A8828583F0D083D08212084D12084D120B
:10084600084D12084DE473E493A3C583C5F0C58330
:10085600C8C582C8F0A3C583C5F0C583C8C582C80C
:01086600226F
:10086700D083D082E493F208740193F20874029360
:09087700F208740393F274047397
:00000001FF
